:10000000283084005830A0008001840AA00B042806
:10001000103095002730960000308E0000308F00A1
:10002000013090000B30970007309F008316FF309F
:10003000850083128316CF30860083120C1D1E2884
:100040000C116400A914A9182915A91C2911A911BA
:1000500029192916291D2912851B2F282912A91AA9
:1000600032282912291E3528A91529192916291DD2
:100070002912051B3C282912A91A3F282912291EDA
:100080004228A915A9192915A91D291129192917C6
:10009000291D2913A91F4D282911291BA917291F1B
:1000A000A913291D58282A185828AB0F5828AC0A1C
:1000B00029192A14291D2A1000302C020319672837
:1000C000A00020092C05A006A01B6C286E2801307A
:1000D0002B02031C6C286E2829116F282915291959
:1000E0008616291D8612A9182915A91C2911861AF8
:1000F0007A282911291D912827302E0203198728D3
:10010000A00020092E05A006A01B8C2890280F30E7
:100110002D02031C8C289028AD0F8F28AE0A2911C0
:1001200095280030AD000030AE00291DAC282730E6
:1001300030020319A228A00020093005A006A01B48
:10014000A728AB280F302F02031CA728AB28AF0F1E
:10015000AA28B00A2911B0280030AF000030B00042
:10016000291DC728273032020319BD28A000200905
:100170003205A006A01BC228C6280F303102031C7E
:10018000C228C628B10FC528B20A2911CB280030D1
:10019000B1000030B200291DD1280030AB00003082
:1001A000AC00A9182915A91C2911861AD8282911CB
:1001B000061EDB282911AA18E1283130B3000030CF
:1001C000B400AA142919F928003034020319EF28C1
:1001D000A00020093405A006A01BF428F82831301F
:1001E0003302031CF428F828B30FF728B40A2915A2
:1001F000FD280030B3000030B400291D1429003060
:10020000360203190A29A00020093605A006A01B02
:100210000F29132931303502031C0F291329B50F7B
:100220001229B60A291118290030B5000030B6008D
:1002300029190616291D0612A9182915A91C291104
:100240000519232929112919A916291DA9128A017D
:100250001E28FF3FFF3FFF3FFF3FFF3FFF3FFF3FA6
:10026000FF3FFF3FFF3FFF3FFF3FFF3FFF3FFF3F9E
:10027000FF3FFF3FFF3FFF3FFF3FFF3FFF3FFF3F8E
:10028000FF3FFF3FFF3FFF3FFF3FFF3FFF3FFF3F7E
:10029000FF3FFF3FFF3FFF3FFF3FFF3FFF3FFF3F6E
:02400E0050035D
:10420000FF00FF00FF00FF00FF00FF00FF00FF00B6
:10421000FF00FF00FF00FF00FF00FF00FF00FF00A6
:10422000FF00FF00FF00FF00FF00FF00FF00FF0096
:10423000FF00FF00FF00FF00FF00FF00FF00FF0086
:10424000FF00FF00FF00FF00FF00FF00FF00FF0076
:10425000FF00FF00FF00FF00FF00FF00FF00FF0066
:10426000FF00FF00FF00FF00FF00FF00FF00FF0056
:10427000FF00FF00FF00FF00FF00FF00FF00FF0046
:10428000FF00FF00FF00FF00FF00FF00FF00FF0036
:10429000FF00FF00FF00FF00FF00FF00FF00FF0026
:1042A000FF00FF00FF00FF00FF00FF00FF00FF0016
:1042B000FF00FF00FF00FF00FF00FF00FF00FF0006
:1042C000FF00FF00FF00FF00FF00FF00FF00FF00F6
:1042D000FF00FF00FF00FF00FF00FF00FF00FF00E6
:1042E000FF00FF00FF00FF00FF00FF00FF00FF00D6
:1042F000FF00FF00FF00FF00FF00FF00FF00FF00C6
:00000001FF
